S01900006F70656E626C745F73746D33326C3437362E73726563F2
S3150800000000800120BD050008490500084D050008C7
S3150800001051050008550500085905000800000000AC
S315080000200000000000000000000000005D05000858
S31508000030610500080000000065050008690500085C
S315080000400D0600080D0600080D0600080D06000836
S315080000500D0600080D0600080D0600080D06000826
S315080000600D0600080D0600080D0600080D06000816
S315080000700D0600080D0600080D0600080D06000806
S315080000800D0600080D0600080D0600080D060008F6
S315080000900D0600080D0600080D0600080D060008E6
S315080000A00D0600080D0600080D0600080D060008D6
S315080000B00D0600080D0600080D0600080D060008C6
S315080000C00D0600080D0600080D0600080D060008B6
S315080000D00D0600080D0600080D0600080D060008A6
S315080000E00D0600080D0600080D0600080D06000896
S315080000F00D0600080D0600080D0600080D06000886
S315080001000D0600080D0600080D0600080D06000875
S315080001100D0600080D0600080D0600080D06000865
S315080001200D0600080D0600080D0600080D06000855
S315080001300D0600080D0600080D0600080D06000845
S315080001400D0600080D0600080D0600080D06000835
S315080001500D0600080D0600080D0600080D06000825
S315080001600D0600080D0600080D0600080D06000815
S315080001700D0600080D0600080D0600080000000020
S30D080001800D0600080D06000833
S3150800018810B5054C237833B9044B13B10448AFF3BB
S3150800019800800123237010BD3000002000000000F5
S315080001A81825000808B5034B1BB103490348AFF3E4
S315080001B8008008BD0000000034000020182500084B
S315080001C801F07CBF01F08ABF08B5054B186910F421
S315080001D8005000D108BD00F035F8012008BD00BF61
S315080001E800080048642000F003B800BF00F006B80D
S315080001F8014B1880704700BF4C00002010B50E4C04
S3150800020801F00AFF236898420ED30C4B1A7862B19C
S315080002184FF09042002020211870916201F0FCFEF0
S31508000228074B1B881844206010BD4FF090420120E8
S31508000238202118709161F1E7500000204E00002037
S315080002484C0000204FF0904320229A62704700BF66
S315080002582C4A136823F0070343F0040310B5136008
S31508000268136803F00703042BFAD12749274B0A68B2
S3150800027822F4C06242F400720A601A6842F4807274
S315080002881A601A685205FCD5586821491F4A20F091
S31508000298F85040F080505860D868014041F4206111
S315080002A841F00201D960D96841F08071D9601968AE
S315080002B841F08071196013689B01FCD59368134C4B
S315080002C843F003039360A36803F00C030C2BFAD1DD
S315080002D8A368104823F0F003A360A36823F4E06337
S315080002E8A360A36823F46053A36001F0E7FA00202B
S315080002F800F0A2F9D4F8883023F00C03C4F8883043
S3150800030810BD00BF002002400070004000100240E7
S315080003188C80FFF900B4C40480B5002492B000F0BC
S31508000328B1F9FFF795FFCDE90C44CDE90E443F4DE9
S315080003381094EB6C3E483F4F43F00403EB64EB6CB8
S3150800034803F004030293029BEB6C43F00103EB648E
S31508000358EB6C03F001030393039BEB6C43F0020376
S31508000368EB64EB6C12AE4FF0904803F0020304936B
S315080003784FF020094FF40053049AC8F8289046F815
S315080003881C3D314600F040FF0123314640460C9398
S31508000398CDF82C90CDE90D440F9400F035FFC6E949
S315080003A80144C6E90344C6E90544CDE908440B9463
S315080003B8AB6D43F40033AB65AB6D03F400330093C0
S315080003C8009BEB6C43F00103EB64EB6C022103F032
S315080003D801030C25019303220723CDE9055140465D
S315080003E805A9DDF804C007920A9300F00DFF4FF43B
S315080003F8E133314638460B93CDE90C44CDE90E4531
S31508000408CDE9104401F0E8F97B6823F490437B6052
S31508000418BB6823F02A03BB603B6843F001033B60D3
S31508000428FFF7CEFEFFF7CEFEFCE700BF001002403E
S3150800043800080048004400400A4B1A6E42F00102C0
S315080004481A661A6E82B002F001020092009A9A6D34
S3150800045842F080529A659B6D03F080530193019B85
S3150800046802B070470010024070B50168184A88B093
S3150800047800239142CDE90333CDE90533079301D02B
S3150800048808B070BD03F1804303F5043311489A6D2B
S3150800049842F000729A659A6D02F000720192019A0A
S315080004A8DA6C42F00202DA64DB6C03F002030293A8
S315080004B80322092303A94FF440750224029ECDE9B5
S315080004C80354CDE9062300F00FFD08B070BD00BF40
S315080004D8006400400004004810B54FF0904400F04E
S315080004E863FF2023A362134800F0F6FD124800F0C4
S315080004F8F3FD204600F0F0FD104B9A6D22F00072CD
S315080005089A659A6D22F400329A65DA6C22F004022A
S31508000518DA64DA6C22F00202DA64DA6C22F0010292
S31508000528DA649A6D22F080529A651A6E22F00102F0
S315080005381A6610BD0008004800040048001002406A
S31508000548704700BFFEE700BFFEE700BFFEE700BF33
S31508000558FEE700BF704700BF704700BF704700BF7F
S3150800056800F0ACB81149124BD1F8882042F4700251
S3150800057810B4C1F888201A68002042F001021A60EF
S3150800058898601A6822F0A85222F410224FF4805470
S315080005981A60DC601A684FF0006422F480221A6038
S315080005A898618C605DF8044B704700BF00ED00E069
S315080005B800100240DFF834D0FFF7D4FF002103E02B
S315080005C80B4B5B58435004310A480B4B42189A4266
S315080005D8F6D30A4A02E0002342F8043B084B9A423B
S315080005E8F9D301F071FFFFF797FEFEE700800120B7
S315080005F830260008000000203000002030000020C7
S315080006086C050020FEE7000010B50A4B4FF0FF32D4
S3150800061800249A63DA639C63DC631A641C649A622E
S315080006289C62DA62DC621A631C63FFF755FF204690
S3150800063810BD00BF0010024038B50F4B1B780BB928
S31508000648012038BD0D494FF47A720546B2FBF3F31B
S315080006580868B0FBF3F000F09DFA04460028EFD1CD
S315080006680F2DEDD8024629464FF0FF3000F05CFA08
S31508000678034B20461D6038BD0400002000000020FA
S315080006880800002000B50C4A136843F4807383B049
S315080006980320136000F036FA0020FFF7CDFF18B1E3
S315080006A8012003B05DF804FB0190FFF7C5FE019829
S315080006B803B05DF804FB00BF00200240034A044B60
S315080006C811681B780B441360704700BF6805002043
S315080006D80400002000287CD038B590F8203004465D
S315080006E8002B73D02268136823F00203136001F005
S315080006F8A1FC054604E001F09DFC401B0A285CD8CD
S3150800070823685A689107F6D41A6842F001021A60F3
S3150800071801F090FC054604E001F08CFC401B0A2811
S315080007284BD823685A68D207F6D5227E012A1A6852
S315080007380CBF42F0800222F080021A60627E012A0B
S315080007481A680CBF42F0400222F040021A60A27EE4
S31508000758012A1A680CBF42F0200222F020021A6009
S31508000768E27E012A1A680CBF22F0100242F0100233
S315080007781A60227F012A1A680CBF42F0080222F082
S3150800078808021A60627F012A1A680CBF42F004023E
S3150800079822F004021A60D4E90221D4E904500A4373
S315080007A861682A43024301390A4301250021DA61AF
S315080007B80846616284F8205038BD636A052243F406
S315080007C800336362012084F8202038BDFFF74CFE09
S315080007D888E70120704700BF90F82030013B012BBD
S315080007E805D9436A43F480234362012070470368A6
S315080007F84869D3F8002242F001022DE9F041CE6992
S31508000808C3F80022012500F01F02D3F81C4205FA96
S3150800081802F2D5432C40C3F81C42B6B3012E15D1B3
S31508000828D3F80C620F68B1F804E0B1F80CC003EB12
S31508000838C00446EA02008E68C3F80C024EEA074767
S315080008484CEA0646C4F84072C4F844628869A0BBF4
S31508000858D3F804022840C3F804020869A8BBD3F8E9
S3150800086814022840C3F81402096A012904D1D3F8E6
S315080008781C120A43C3F81C22D3F8002222F00102EC
S31508000888C3F800220020BDE8F081D3F80C72CE68C0
S31508000898B1F804C00C8803EBC00805EA07008F689E
S315080008A8C3F80C0288694CEA064644EA0744C8F8BD
S315080008B84062C8F844420028CAD0D3F80402104354
S315080008C8C3F8040208690028C9D0D3F814021043EB
S315080008D8C3F81402C8E700BF38B590F82030012BD2
S315080008E805D0436A43F400234362012038BD0268F1
S315080008F8022380F82030136823F0010313600446A6
S3150800090801F098FB054604E001F094FB401B0A2811
S3150800091807D823685B6813F00103F5D163621846A4
S3150800092838BD636A052243F400336362012084F8FC
S31508000938202038BD70B490F820400568013C012C89
S31508000948AE6806D9436A43F480234362012070BC23
S31508000958704716F0E05F2ED0C6F30166032E31D035
S315080009680120B04018608B6893BB0C68C86806F10C
S3150800097818031B0140EA4450E850087D0969360106
S31508000988AB190128C3F8841105D1D3F8841141F4A9
S315080009988071C3F8841135445168C5F88C111268FA
S315080009A8C5F88821D3F8802142F001020020C3F84F
S315080009B8802170BC7047436A43F40013436270BCD5
S315080009C801207047436A43F4000343620120BEE7E7
S315080009D8C8684C68034306F11800000143EAC403D3
S315080009E82B50CAE790F82030013B012B01D900208B
S315080009F8704703689B68890631EA030314BF012018
S31508000A08002070472DE9F04190F82040013C012C60
S31508000A1806D9436A43F4802343620120BDE8F0817E
S31508000A280568002958D02C69A40758D00C012E1936
S31508000A38D6F8B07107F004079760002F5CD1D6F88E
S31508000A48B0717F0D1760D6F8B0E1D6F8B4C1D6F8FC
S31508000A58B471D6F8B46125440EF0020ED5F8B881FB
S31508000A68C7F307270CF00F05360CC2E903E5C2E9F8
S31508000A78056783F8008002682244D2F8B821120A6A
S31508000A885A7002682244D2F8B821120C9A70026881
S31508000A982244D2F8B821120EDA7002682244D2F833
S31508000AA8BC211A7102682244D2F8BC21120A5A716A
S31508000AB802682244D2F8BC21120C9A7102681444BE
S31508000AC8D4F8BC21120EDA71026879B9D36843F0F2
S31508000AD820030846D360A1E7EC68A607A6D1436AAF
S31508000AE843F4001343620120BDE8F081136943F01B
S31508000AF820031361002091E7D6F8B071FF08576004
S31508000B08A1E700BF074AD3684FF6FF010B4000026A
S31508000B1843F0BF6300F4E06043F400330343D36053
S31508000B28704700BF00ED00E0184BDB68C3F30223EB
S31508000B3830B4C3F10705042D03F1040428BF0425BE
S31508000B48062C19D9033B4FF0FF349C4022EA0404CB
S31508000B584FF0FF32AA4021EA020101FA03F22243C2
S31508000B6812010028D2B20ADB00F1604000F56140A4
S31508000B7880F8002330BC704700242346E8E7044B76
S31508000B8800F00F0003441A7630BC704700ED00E009
S31508000B98FCEC00E00138B0F1807F0ED2084B10B4A7
S31508000BA8084C5860F02084F82300002207211046D4
S31508000BB89A6019605DF8044B70470120704700BFBA
S31508000BC810E000E000ED00E0064B5A69002A01DB58
S31508000BD8002070470449054A99609A605869C00F09
S31508000BE8704700BF0020024023016745AB89EFCD57
S31508000BF8034A536943F0004353610020704700BF16
S31508000C080020024070B5054601F014FA114C064654
S31508000C1801E06A1C0FD12369DB03FAD423694CF275
S31508000C28FA3213400ED1206910F0010002D00122D1
S31508000C381846226170BD01F0FDF9801BA842EAD367
S31508000C48032070BD04494A681A434A600120236193
S31508000C5870BD00BF002002400C0000202DE9F843B3
S31508000C68344E96F800C0BCF1010F35D098460746B1
S31508000C7801234CF2503014460D463370FFF7C2FF75
S31508000C88814620B1002333704846BDE8F8832A4ACE
S31508000C987060136813F4806323D01368022123F461
S31508000CA8806313603177FFB9234A536943F0010318
S31508000CB853612C60BFF36F8F4CF25030C5F804802F
S31508000CC8FFF7A0FF6FF0010181461B4A53690B40E5
S31508000CD8536100F051F8D5E74FF002094846BDE8D8
S31508000CE8F8833377002FDFD07B1E012B05D94CF20A
S31508000CF85030FFF787FF8146EBE70F494B6943F406
S31508000D08802322464B61EFF3108072B6291B04F53F
S31508000D1880741368535004329442FAD180F31088C9
S31508000D28022F4CF25030E4D1FFF76CFF6FF48021A4
S31508000D388146CAE70C000020002002400D4A536984
S31508000D48C9074CBF23F4006343F400635361094B96
S31508000D585A69C00022F4FF6200F4FF601043586124
S31508000D685A6942F002025A615A6942F480325A6153
S31508000D78704700BF0020024013490B7FDBB203F01F
S31508000D88FD02012A0CD1114A106840F4006010606F
S31508000D98106820F400601060106840F40070106055
S31508000DA8023B012B0CD8094B1A6842F480521A6088
S31508000DB81A6822F480521A601A6842F480621A6025
S31508000DC800230B77704700BF0C0000200020024064
S31508000DD82DE9F047414E3378012B4AD004460125C0
S31508000DE84CF2503088463570FFF70CFF074620B19D
S31508000DF8002333703846BDE8F087394B70601A68A7
S31508000E0812F4007F1A6838D1510565D51A68022187
S31508000E1822F480621A6031772368012B3AD04FF0A2
S31508000E28FF33C8F80030D4E902532B449D421DD23B
S31508000E38DFF8ACA0DFF8AC9005E0D4E9023201355A
S31508000E481344AB4212D961682846FFF777FF4CF27C
S31508000E585030FFF7D7FEDAF8143003EA0903CAF860
S31508000E6814300028E9D0C8F800500746FFF784FF71
S31508000E78BEE702273846BDE8F08722F400721A60F2
S31508000E881A68500526D51A68032122F480621A6062
S31508000E983177C1E76368DA0704D511494A6942F028
S31508000EA804024A619B0704D50D4A536943F4004373
S31508000EB853610B4C636943F4803363614CF25030D9
S31508000EC8FFF7A0FE636923F4004323F004030746EB
S31508000ED86361CBE735779FE730779DE70C000020FD
S31508000EE80020024005F8FFFF2DE9F04FD1F80090E1
S31508000EF883B0B9F1000F00F0B180DFF8D8B18846A1
S31508000F080025012303FA05F717EA090A00F0A18064
S31508000F18D8F8043023F010016C0003220139A240E6
S31508000F2801296FEA02020ED88668D8F80C1016400E
S31508000F38A140314381604668C3F3001126EA0706D3
S31508000F48A94031434160D8F8086003F00301032932
S31508000F5806FA04F600F08580C76817403E43022B58
S31508000F68C66040F08D804FEAD50E00EB8E0E05F070
S31508000F780707DEF82060BF004FF00F0C0CFA07FCD5
S31508000F8826EA0C0CD8F81060BE4046EA0C06CEF8DD
S31508000F9820600668A14032401143DA00016058D53E
S31508000FA845490A6E42F001020A660A6E25F00304EC
S31508000FB804F1804402F0010204F58034019205F038
S31508000FC803020199A66892000F219140B0F1904F4B
S31508000FD826EA010116D0394EB04259D0384EB042E9
S31508000FE851D0384EB0425DD0374EB0425FD0374EFA
S31508000FF8B04252D0364EB0420CBF0626072606FA2D
S3150800100802F21143A160DBF800206FEA0A01DF0348
S3150800101854BF0A404AEA0202CBF80020DBF804204B
S315080010289E0354BF0A404AEA0202CBF80420DBF8BA
S315080010380820DC0254BF0A404AEA0202CBF8082014
S31508001048DBF80C209B0254BF0A404AEA0202CBF896
S315080010580C20013539FA05F37FF453AF03B0BDE820
S31508001068F08FD0F82CC0C3F3C00E2CEA070C7746CD
S31508001078AF4047EA0C07C762C76817403E43C660D1
S31508001088122B86D16FE7022606FA02F21143B9E750
S31508001098012606FA02F21143B4E7052606FA02F211
S315080010A81143AFE7032606FA02F21143AAE7042614
S315080010B806FA02F21143A5E70010024000040048A8
S315080010C800080048000C00480010004800140048B2
S315080010D80018004800040140B0F1904F16D0424B62
S315080010E898423AD0414B98421BD0414B984242D03D
S315080010F8404B98424DD0404B984220D03F4B98429F
S3150800110855D03F4B984260D0012070473D4BDA6A6C
S3150800111842F00102DA62DA6A22F00102DA62002093
S31508001128704703F1784303F502330020DA6A42F080
S315080011380402DA62DA6A22F00402DA62704703F114
S31508001148784303F5FE330020DA6A42F02002DA62B1
S31508001158DA6A22F02002DA62704703F1784303F567
S3150800116803330020DA6A42F00202DA62DA6A22F007
S315080011780202DA62704703F1784303F50133002067
S31508001188DA6A42F00802DA62DA6A22F00802DA62F1
S31508001198704703F1784303F500330020DA6A42F012
S315080011A81002DA62DA6A22F01002DA62704703F18C
S315080011B8F82303F580330020DA6A42F04002DA623F
S315080011C8DA6A22F04002DA62704703F1784303F5D7
S315080011D8FA330020DA6A42F08002DA62DA6A22F022
S315080011E88002DA62704700BF000400480008004819
S315080011F8000C004800100048001400480018004871
S31508001208001C0048001002402DE9F0470D6895FAC1
S31508001218A5F44E68B4FA84F435FA04F306F1FF3CEB
S3150800122874D001274FF00F084FF0030E2EE0B2FADC
S3150800123882F2520006FA02F242EA0902BCF1010FEA
S31508001248026071D90A69D0F80CA093FAA3F9B9F122
S31508001258000F07D0B9FA89F94FEA49090EFA09F9C8
S315080012682AEA090A93FAA3F9B9F1000F24D0B9FAB8
S3150800127889F94FEA490902FA09F242EA0A02022EEC
S31508001288C26022D0013435FA04F33FD007FA04F3D2
S315080012982B40F7D0D0F8009093FAA3F232B1B2FAFD
S315080012A882F252000EFA02F229EA020993FAA3F226
S315080012B8002ABCD14022BDE74FF0400902FA09F2DC
S315080012C842EA0A02022EC260DCD1FF2BD1F814903A
S315080012D84CD8026A93FAA3FABAF1000F07D0BAFAF9
S315080012E88AFA4FEA8A0A08FA0AFA22EA0A0293FAEC
S315080012F8A3F3002B56D0B3FA83F39B0009FA03F33A
S3150800130813430134036235FA04F3BFD1BCF1010F64
S3150800131807D8CA68436802FB05F223EA0505154398
S3150800132845600020BDE8F0878A68D0F808A093FAD7
S31508001338A3F9B9F1000F07D0B9FA89F94FEA4909AB
S315080013480EFA09F92AEA090A93FAA3F9B9F1000F74
S3150800135809D0B9FA89F94FEA490902FA09F242EABB
S315080013680A0282606EE74FF04009F6E71B0A426AEE
S3150800137893FAA3FABAF1000F07D0BAFA8AFA4FEA2B
S315080013888A0A08FA0AFA22EA0A0293FAA3F33BB186
S31508001398B3FA83F39B0009FA03F31A43426271E727
S315080013A88023F8E78023A9E710B4284B1A6842F087
S315080013B8010283B01A601A689207FCD5196824488E
S315080013C8224A21F0F00141F060011960596821F4B8
S315080013D87F415960596821F0F85141F0805100243D
S315080013E859609C6019680191019908400190019912
S315080013F821F080610191019921F0805101910199AB
S315080014081960106810F02850FBD14FF48053D36048
S3150800141813615361136840F23F3123F48023136044
S3150800142890610191019B43F040030193019B43F0AE
S3150800143880030193019B1362D2F8943043F40003A6
S31508001448C2F8943003B05DF8044B704700100240A8
S31508001458FFF4FEFE1E4AD36803F00303022B2BD0C3
S31508001468032B14D0136813F008030BD013681B0753
S3150800147824D4D2F894301B0903F0F003154A52F81D
S31508001488231005E0116809071CD51268F6E7124902
S315080014980F4BDA68D868DB68C3F34163C2F30212F4
S315080014A8C0F3062001335B000132B1FBF2F200FB00
S315080014B802F0B0FBF3F070470849E9E71368C3F38D
S315080014C80313DBE7D2F89430C3F30323D6E700BF48
S315080014D8001002404825000800127A000024F4008B
S315080014E81E4B9B6803F00C030C2B08D8DFE803F0A7
S315080014F80707070714070707160707071800174AED
S31508001508136813F008030DD1116809071DD5126869
S31508001518134A52F823007047124870471248704712
S31508001528FFF798BF13681B0708D4D2F894300C4AFB
S315080015381B0903F0F00352F8230070471368084A9A
S31508001548C3F3031352F823007047D2F89430044AB9
S31508001558C3F3032352F82300704700BF0010024064
S31508001568482500080024F40000127A0038B5044615
S31508001578FFF7B6FF0B4B20609A680B4D0B49C2F371
S315080015880312AA5CD04060609A68C2F302228A5C99
S3150800159820FA02F2A2609B68C3F3C223CB5CD84048
S315080015A8E06038BD001002403025000840250008D4
S315080015B8032810B52ED00C2803D0302849D000208F
S315080015C810BD4C4BD3F8883003F00C0343F4402382
S315080015D8A3F540230C2BF2D801A252F823F000BF3A
S315080015E8B5160008C7150008C7150008C715000866
S315080015F88F160008C7150008C7150008C71500087C
S31508001608A5160008C7150008C7150008C715000855
S31508001618D5160008374C384AD4F8883003F003033F
S3150800162843F44033934232D0B3F1031F22D0013A30
S31508001638934228D0FFF754FFA368A2682F4C304975
S31508001648C3F30313C2F3C222E35C8A5CD840D040D2
S3150800165810BD284C2B4AD4F8883003F0300343F4DD
S31508001668401393420FD03BD9274A93420FD0B3F180
S31508001678301FA4D1D4F8903013F0020F0CBF002005
S315080016884FF4004010BDBDE81040FFF729BF236896
S315080016981E4813F4806F08BF002010BD154B1B4861
S315080016A81B6813F4806F08BF002010BDFFF718FFEA
S315080016B8104A124C936892681149C3F30313C2F38C
S315080016C80222E35C8A5CD840D04010BD094BD3F8A7
S315080016D8903013F0020F0CBF00204FF4004010BDE5
S315080016E8B3F5401F7FF46BAFFFF7FAFEA368A2684D
S315080016F8024CE1E70010024002000300302500080A
S315080017084025000810003000200030000024F400AE
S31508001718C02810B51CD0B0F5407F2AD1264C274AD8
S31508001728D4F8883003F4407343F0407393423FD0AB
S3150800173821D9234A934234D0B3F1032F19D1D4F8C7
S31508001748903013F0020F0CBF00204FF4004010BD74
S31508001758194C1C4AD4F8883003F0C00343F44003F4
S31508001768934225D019D9184A93421AD0B3F1C01F03
S31508001778E5D0002010BDB3F1407FFAD1FFF7B0FEDF
S31508001788A368A268114C1249C3F30313C2F30222D1
S31508001798E35C8A5CD840D04010BDB3F5400FEDD065
S315080017A8E7E723680B4813F4806F08BF002010BDCD
S315080017B8BDE81040FFF794BE001002400001000380
S315080017C8000200034000C0008000C0003025000861
S315080017D8402500080024F4000368DB072BD470B5FD
S315080017E8D1E9032604464B6888690D4613432168E0
S315080017F82C4A33430A400343134323606268AB68A1
S315080018086869294922F440521A436260A36823F496
S31508001818407303438C42A3600FD0244B9C4221D0CB
S31508001828234B9C4222D0234B9C4223D0224B9C42DA
S3150800183824D0012070BD012070470320FFF7B8FEA9
S315080018480028F6D02B68002BF3D0A969B1F5004F0C
S315080018584FEA530217D01044B0FBF3F080B2E060A9
S31508001868002070BD0C20FFF7A3FEE9E73020FFF73C
S315080018789FFEE5E7C020FFF74BFFE1E74FF440700E
S31508001888FFF746FFDCE74FF6F07102EB4000B0FBC6
S31508001898F3F000EA0103C0F342001843E0600020B1
S315080018A870BD00BFF369FFEF0038014000440040EF
S315080018B800480040004C004000500040014B1860AA
S315080018C8704700BF0000002072B6704762B67047BE
S315080018D8F0B58BB06846FFF749FE02982A4B2B4AA3
S315080018E8A3FB0030800902F1220C022405260025F4
S315080018F84FF4FA7702E09678D4780232331903FB64
S315080019080773B0FBF3F103FB110323B98DB26B1E02
S31508001918B3F5806F33D39445EDD1AC211C481D4CE3
S315080019281D4E00F095FB1D4F1D4B7C617D60002404
S31508001938012538463B603C767C76BC763C777C77D6
S31508001948C7E902443E61FD76FEF7C4FE4CF6E0435D
S3150800195804226946CDE9054401940494009338465F
S315080019680E234FF6E074CDE90242099307950895C8
S31508001978FEF732FF3846FEF7AFFF0BB0F0BD013E63
S31508001988013C36042405CEE7D34D6210B425000879
S31508001998782500080000F0FF0000FFFF540000202B
S315080019A80064004030B589B00246069140F2E175F8
S315080019B8002401AB02A90E480295CDE90444FEF7B6
S315080019C8B9FF08B109B030BD00F026FB084C00F194
S315080019D8320505E000F000FC00F01EFBA842F1D82D
S315080019E801992046FEF7FEFF0028F3D109B030BD5D
S315080019F85400002010B588B00C46034601AA0021F9
S31508001A080A48FEF7FFFF70B9019A40F267639A42DF
S31508001A1801D008B010BD039B002BFAD1059B237093
S31508001A28012008B010BD002008B010BD54000020E1
S31508001A38FFF74ABF10B500F01BFA00B910BDFEF74C
S31508001A48C3FB0028FAD000F091FBFEF7DDFD00F095
S31508001A58CDFA00F00FFA074B20F0604020F07F001F
S31508001A68986000F007FA4468FFF730FF2346BDE898
S31508001A781040184700ED00E072B170B5551EADB2BA
S31508001A880D440C460135461A2378A355013400F04F
S31508001A98A3FBAC42F8D170BD704700BF2DE9F843E7
S31508001AA88046FFF791F81A4B4FF4004208F10409EB
S31508001AB81A61002408E0D5E90023BB4208BFB242F0
S31508001AC81AD1B4F5007F1DD009EB0403D3E90067E2
S31508001AD8D8F80050254400F07FFB32463B46294695
S31508001AE80020FFF7BBF808340028E4D00024FFF7E5
S31508001AF87FF82046BDE8F8830446FFF779F82046BC
S31508001B08BDE8F8830124FFF773F82046BDE8F88393
S31508001B180020024070B50F4CA0420D4615D00E4B5A
S31508001B2899420CD123689D4207D02046294640F899
S31508001B38045B4FF40072FFF79FFF204670BD064608
S31508001B48FFF7ACFF18B13446ECE7044CEAE704465D
S31508001B58F3E700BF80020020002800087C00002068
S31508001B682DE9F8430C46016824F4FF781D464B1CFA
S31508001B780746164628F0010833D0884526D1043486
S31508001B88641A3C4408F5007807F1040905E016F8D4
S31508001B98013B04F8013B013D15D000F01DFBA4EB01
S31508001BA80903B3F5007FF2D338464146FFF7B2FF7B
S31508001BB8074698B100F104094C4616F8013B04F8A3
S31508001BC8013B013DE9D10120BDE8F8833846414685
S31508001BD8FFF7A0FF074608B10168D0E70020BDE86F
S31508001BE8F8838146414649F8048B4FF40072484603
S31508001BF8FFF742FF3968C0E70349044A4FF0FF3345
S31508001C080B601360704700BF7C000020800200202C
S31508001C18104B30B44D1E1C1AA54213D80E4CA042C0
S31508001C2810D9441E0C449C420CD820F4FF730B4C64
S31508001C3823F00103A3420B46014606D0084830BCE8
S31508001C48FFF78EBF002030BC7047064830BCFFF748
S31508001C5887BF00BFFFFF0F08FF27000800280008F6
S31508001C687C000020800200202DE9F0413F4B4C1EE5
S31508001C781A1A944286B06AD820F4FF683C4A28F0B3
S31508001C880708904563D9421E0A449A425FD80D1838
S31508001C98A5EB0805C5F30A03C5F3CF250BB101352E
S31508001CA8ADB2FEF791FF33494FF4004000220123F5
S31508001CB8086102920593002D4ED0013DABB208F596
S31508001CC800652D4C2D4F2E4E05EBC32515E0914288
S31508001CD81ABF06EA432303F100633B46984534BF17
S31508001CE80123022301A902A80393FFF771F8002824
S31508001CF839D108F50068A8452ED000F06DFA236892
S31508001D084FF6FF7299B291421ABF06EA432303F1C6
S31508001D1800633B46984534BF08F17843A8EB0303AC
S31508001D28DB0A184A0493136813F4807F23684FF66E
S31508001D38FF7299B2CBD091421ABF06EA432303F140
S31508001D4800633B46984534BF02230123CAE70024AB
S31508001D58204606B0BDE8F0810124FEF749FF204673
S31508001D6806B0BDE8F0810024F7E700BFFFFF0F08BB
S31508001D78FF27000800200240E075FF1F000008083A
S31508001D8800FEFF01000001400F4A1368013318D00E
S31508001D9830B5D2E90135D2E903012B440344546925
S31508001DA80A480B44D2E90612234483B00B44134469
S31508001DB802AA5B4242F8043D0421FFF729FF03B053
S31508001DC830BD0120704700BF80020020882900081E
S31508001DD80E4A0F4B0F4912680F481B68096830B43A
S31508001DE80E4C05682468134408300B440C490068EF
S31508001DF80C4A096812682B44234403440B44D3420B
S31508001E080CBF0120002030BC704700BF002800081E
S31508001E1804280008082800080C28000810280008C4
S31508001E2818280008882900080A4808B503680133ED
S31508001E380BD109480368013305D0FFF72FFE003098
S31508001E4818BF012008BD012008BDFFF727FE002896
S31508001E58EFD108BD800200207C00002000487047AA
S31508001E6800280008FFF7C8BEFFF7D2BEFFF7FCBE7A
S31508001E78FFF7AEBFFFF7F2BF08B5FFF785FF00B952
S31508001E8808BDBDE80840FFF7CFBF00BF38B5084C06
S31508001E98208500F0C1F800F10A0505E000F09CF974
S31508001EA800F0BAF8A84202D8E3691B06F6D538BD89
S31508001EB80044004030B50D4C236889B023F001036F
S31508001EC823600C22002320464FF4614501A9CDE979
S31508001ED80153CDE90333CDE906330592FFF77CFCB8
S31508001EE8236843F00103236009B030BD004400406D
S31508001EF8402938B50D46044611D82846ADB2FFF72D
S31508001F08C5FF5DB1013D14FA85F5013C00F064F999
S31508001F1814F8010FFFF7BAFFAC42F7D138BD77219D
S31508001F28014800F095F8E8E7D8250008F8B51F4DE8
S31508001F382C786CB91E4BDA69920606D59B8C1D4916
S31508001F48DBB25A1E3F2A0B7026D900242046F8BD54
S31508001F58174AD46914F0200415D0174C978C23789F
S31508001F680E461449CA18013357700A78DBB29A42E2
S31508001F782370EAD10131FFF77FFD237833700023F8
S31508001F882B700124E2E700F047F80C4B1B68643312
S31508001F989842DAD92C70D9E700F03EF8074B064A7A
S31508001FA81860012314702B70D0E700BFC504002001
S31508001FB80044004084040020C6040020C804002009
S31508001FC8074B084910B40022074C1A6005205A60C6
S31508001FD89A605C609A605DF8044B18600A607047FE
S31508001FE810E000E0CC0400207F380100024B0022F4
S31508001FF81A605A609A60704710E000E0044B1B6844
S31508002008DB0303D5034A136801331360704700BF1F
S3150800201810E000E0CC040020044A054B1268186852
S31508002028D20344BF01301860704700BF10E000E0D3
S31508002038CC040020044A054B12681868D20344BF2A
S3150800204801301860704700BF10E000E0CC0400209B
S3150800205808B500F0C1F8FCE710B500F0B3F8012898
S3150800206803D00B4C2378012B00D010BDFFF7D4FF03
S31508002078084B094A1B681268134403F5FA73984211
S31508002088F3D300232370BDE81040FFF7D3BC00BF85
S31508002098D4040020D0040020D804002008B5054B35
S315080020A801221A70FFF7B8FF034B1860BDE808400D
S315080020B8FFF7D2BFD4040020D804002008B5FFF7DC
S315080020C8B7FC00F087F8FFF77BFFFFF7CBFE00F0B9
S315080020D811F8BDE80840FFF7E1BF00BF08B500F0F2
S315080020E87BF8FFF78BFF00F015F8BDE80840FFF707
S315080020F8B3BF00BF10B5064C00F070F8FFF7E8FB51
S3150800210801232370FFF7D6FE0023237010BD00BFF6
S315080021182C00002000B583B00DF107011148FFF720
S3150800212869FC012814D00DF107010E48FFF7FEFED9
S31508002138012802D003B05DF804FB0B4B9DF8071085
S31508002148084800221A7000F065F803B05DF804FB29
S31508002158054A9DF8071003460248137000F05AF816
S31508002168E1E700BFDC0400202C000020704700BF10
S3150800217870B50A4C2378012B0D46064608D01BB9BC
S31508002188E9B23046FFF7B4FEBDE8704000F03AB849
S31508002198C9B2FFF707FC2378F1E700BF2C00002037
S315080021A8054B1B78013BDBB2022B9ABF034A32F870
S315080021B813004020704700BF2C000020182600088E
S315080021C8FFF7EEBF08B500F015F8003018BF012074
S315080021D808BD00BFFEF706B8FEF708B8044B00228C
S315080021E89A6483F84320A3F844201A809A707047A3
S315080021F81C050020024B1878003018BF01207047CC
S315080022081C050020024B002283F84320704700BFB4
S315080022181C050020F8B50378A74CFF2B40D0227878
S31508002228012A00D0F8BDC93B0546352B00F22B819B
S31508002238DFE813F0BC00290129017A0029012901E0
S31508002248D20067008800940029012901290129017B
S315080022582901290129012901290129012901290118
S315080022682901290129012901290129012901290108
S3150800227829012901290129012901290129012901F8
S315080022882901290129012901A300DD00EA00FE0028
S315080022982901290129010601290115011D01D50070
S315080022A8102100220125E370217162712580FFF74C
S315080022B877FFA071FFF784FFE071FFF781FF082316
S315080022C8D84020726572A572A4F84430FFF7CAFD93
S315080022D894F84330012B05D0B4F944100029A1DD40
S315080022E889B206E0FE2210230221E2702371A4F8BF
S315080022F84410012384F843307048BDE8F840FFF7D6
S3150800230837BFFFF74DFF6B780138984274DDFF2217
S315080023180123E270A4F844306978002940F0BF80A8
S31508002328FFF7AAFD0028D3D1FE2131220223E17046
S315080023382271A4F8443094F84330012BD2D0B4F86B
S315080023484410D6E74168A06CFFF790FD0028EBD04B
S31508002358FF220123E270A4F84430ECE70025FF23A6
S31508002368E37025716571FFF71BFF0723A071E571F7
S3150800237825726572A4F84430DDE7FF23E3704568E3
S31508002388A66C4DB17719002516F8013B1D44FFF7D1
S3150800239823FFB742EDB2F7D1012100220823C4F87A
S315080023A80750A180A271A4F84430C4E7A66CFFF7C9
S315080023B8F7FE6A1C411E3046FFF756FD0028B3D0C3
S315080023C8FF23E370FFF7ECFEA36C013803440122F0
S315080023D8A364A4F84420AEE7FFF72CFBB8E700216E
S315080023E8FF2201232180E270A4F84430A3E7FFF70F
S315080023F8D7FE6B7883424ED3FE2122220223E17050
S315080024082271A4F8443096E7FFF7CAFE6A78904224
S31508002418F2D9A16C2A48FFF72FFBFF23E3706A78E5
S31508002428A36C1344A3646B780133A4F844304FE7CC
S31508002438FF23E3704368A3640123A4F844307AE7CA
S31508002448FF232048E370072100230822A06423718C
S315080024586371A371C4F80710A4F844206BE7FE213A
S3150800246800220223E1702271A4F8443063E7FF22B0
S3150800247800236178E27006222371E3802372617172
S31508002488A4F8442057E7FE2120220223E17022718E
S31508002498A4F844304FE76968A1646A78BAE7AA1CC1
S315080024A8A06CFFF7E1FC00283FF43EAF6A78A36CFE
S315080024B81344A3640CE700BF1C0500201F05002071
S315080024C8200500202026000870B50D4E0D4CA41BCB
S315080024D8A4100025A54209D10B4E0C4C00F018F89B
S315080024E8A41BA4100025A54205D170BD56F82530B1
S315080024F898470135EEE756F8253098470135F2E74B
S315080025082826000828260008282600082C26000859
S31508002518F8B500BFF8BC08BC9E467047F8B500BFBA
S30D08002528F8BC08BC9E4670478A
S315080025300000000000000000010203040607080965
S315080025400000000001020304A0860100400D0300FC
S31508002550801A060000350C0040420F0080841E00D9
S3150800256000093D0000127A000024F40000366E01CE
S315080025700048E801006CDC02433A2F576F726B2F54
S31508002580736F6674776172652F4F70656E424C542F
S315080025902F5461726765742F536F757263652F4187
S315080025A0524D434D345F53544D33324C342F63618F
S315080025B06E2E6300050206020603070308030903D5
S315080025C009040A040B040C040C050D050E050F0579
S315080025D00F06100610071008433A2F576F726B2F15
S315080025E0736F6674776172652F4F70656E424C54CF
S315080025F02F5461726765742F536F757263652F4127
S31508002600524D434D345F53544D33324C342F72730D
S315080026103233322E6300000008000000000000007C
S30D080026204F70656E424C540030
S30908002628AD010008EA
S3090800262C890100080A
S3150800263000093D0001000000100000000000000035
S31508002640000000000000000000000000010000007B
S315080026500000000000000000000000000400000068
S705080005BD30
